:020000040000FA
:10000000831285010730990083169F01EF30850028
:100010008312A00148200000A00A20080F39031D08
:10002000013082071A2814285A30212005164A2048
:1000300005120A282430212005163A302120051205
:100040000A28F13EA10021182528A1182728A11867
:100050002928FC3E031829280800FF3EA2005E3034
:10006000212060302120A20B31280800FF3EA30090
:1000700063302D205D30212063302D205F30212022
:10008000A30B3C2808004720482048204720482050
:080090004B20000000000800F5
:02400E00D33F9E
:00000001FF
